:020000040800F2
:10000000D00D002439030008F1080090A3080090E7
:10001000450300083D0100904310009000000000DF
:10002000000000000000000000000000F508009043
:100030003F01009000000000F3080090F7080090D6
:100040005303000853030008530300085303000838
:1000500053030008530300084101009053030008B4
:100060004F0100905501009053030008530300080E
:100070005303000853030008530300085303000808
:1000800053030008530300085303000853030008F8
:1000900053030008530300085303000853030008E8
:1000A00053030008530300085303000853030008D8
:1000B00053030008530300085303000853030008C8
:1000C00053030008530300085303000853030008B8
:1000D0005303000891140008530300085303000859
:1000E000470100905303000800000000530300087C
:1000F0005303000853030008530300085303000888
:100100005303000853030008530300085303000877
:100110005303000853030008530300085303000867
:100120005303000853030008530300085303000857
:100130005303000853030008530300085303000847
:1001400000000000000000000000000000000000AF
:100150005303000853030008530300085303000827
:100160005303000853030008530300085303000817
:100170005303000853030008530300085303000807
:1001800053030008530300085303000853030008F7
:1001900053030008530300085303000853030008E7
:1001A00053030008530300085303000853030008D7
:1001B00053030008530300085303000853030008C7
:1001C00053030008530300085303000853030008B7
:1001D00053030008530300085303000853030008A7
:1001E0005303000853030008530300085303000897
:1001F0005303000853030008530300085303000887
:100200005303000853030008530300085303000876
:100210005303000853030008530300085303000866
:1002200053030008530300085303000800000000B4
:1002300053030008530300080000000053030008A4
:100240005303000853030008530300085303000836
:100250005303000853030008530300085303000826
:100260005303000853030008530300085303000816
:100270005303000853030008530300080000000064
:1002800053030008000000005303000800000000B2
:10029000000000005303000800F002F800F03CF8F2
:1002A0000AA090E8000C82448344AAF10107DA45D1
:1002B00001D100F031F8AFF2090EBAE80F0013F0E7
:1002C000010F18BFFB1A43F0010318474C1300003D
:1002D0006C130000103A24BF78C878C1FAD85207CE
:1002E00024BF30C830C144BF04680C6070470000B0
:1002F0000023002400250026103A28BF78C1FBD82F
:10030000520728BF30C148BF0B6070471FB501F0CE
:1003100075F91FBD10B510BD00F0AAF81146FFF722
:10032000F5FF01F025F900F0C8F803B4FFF7F2FF7C
:1003300003BC01F0DFF80000094880470948004786
:10034000FEE7FEE7FEE7FEE7FEE7FEE7FEE7FEE785
:10035000FEE7FEE704480549054A064B70470000E2
:100360000D14000899020008D0010024D00D0024CB
:10037000D0030024D0030024704753EA020C00F09D
:1003800069802DE9F04B4FF00006002B1FBFB3FA38
:1003900083F503FA05F424FA05F65E4012BF16430E
:1003A000B2FA82F502FA05F4C5F120051EBF22FA61
:1003B00005FC44EA0C04203556EA044C4FEA144488
:1003C00018BF641C4FF000084FF00009904271EB19
:1003D000030C39D3002919BFB1FA81F701FA07F6E6
:1003E000B0FA80F700FA07F6C7F120071EBF20FA1F
:1003F00007FC46EA0C062037B6FBF4FCA7EB050722
:10040000103F07F01F0BCBF120060CFA0BFB2CFA68
:1004100006F644BFB3460026202FA4BF5E464FF029
:10042000000B5BEA060C08BF4FF0010B19EB0B0940
:10043000ABFB027C48EB0608C01B06FB02CC0BFBA7
:1004400003CC71EB0C01C1E70B460246414648461E
:10045000BDE8F08B13B54FF000004FF00001AFF393
:100460000080BDE81C407047704770477047704778
:10047000754600F02BF8AE4605006946534620F05D
:100480000700854618B020B5FFF764FFBDE820409F
:100490004FF000064FF000074FF000084FF0000B40
:1004A00021F00701AC46ACE8C009ACE8C009ACE8F3
:1004B000C009ACE8C0098D46704710B50446AFF3DB
:1004C00000802046BDE81040FFF72FBF004870476E
:1004D0006C01002440F2B52CC9F2000C604740F2D8
:1004E000A93CC9F2000C604740F2116CC9F2000C43
:1004F000604740F2056CC9F2000C604740F2FB7C9B
:10050000C9F2000C604740F6A50CC9F2000C604728
:1005100040F25D1CC9F2000C604740F2010CC9F2C8
:10052000000C604740F2917CC9F2000C604700006B
:10053000F0B5BFF34F8FBFF36F8F1D4900200860E8
:10054000BFF34F8FBFF36F8F1A4C216841F4003116
:100550002160BFF34F8FBFF36F8F16497031086072
:10056000BFF34F8F081F006843F6FF75104E10361B
:10057000C0F34E31C0F3C90305EA4112184642EAFE
:1005800080773760401EFAD2491EF5D2BFF34F8FF5
:10059000206840F480302060BFF34F8FBFF36F8F2F
:1005A00003484C30016841F004010160F0BD0000D7
:1005B00050EF00E014ED00E00248016841F0010155
:1005C00001607047200400584FF0B04110B5D1F8D9
:1005D0008820024203D0C1F88800FFF77BFF10BDDE
:1005E0002DE9F84F6C4C00224FF0B04A4FF0010B50
:1005F0004FF0030E4FF00F090B680BFA02F73B4068
:10060000BB4270D14D68022D01D0122D12D1D508F8
:1006100000EB850CDCF820605507ED0E09FA05F8B3
:1006200026EA0806D1F8108008FA05F848EA060814
:10063000CCF82080D0F80080560091F804C00EFA63
:1006400006F50CF0030C28EA05080CFA06FC4CEA47
:10065000080CC0F800C0D1F804C0BCF1010F08D0EC
:10066000BCF1020F05D0BCF1110F02D0BCF1120F8A
:1006700016D1D0F808C0D1F80C802CEA050C08FA85
:1006800006F848EA0C08C0F80880D0F804C02CEA44
:10069000070C0F79C7F30017974047EA0C0747602C
:1006A000C768AF438D68B5403D43C5604D68ED00F8
:1006B0006BD53A4D2E6846F002062E602D6822F06A
:1006C000030606F1B04605F002050095D6F808C409
:1006D00095072F0F09FA07F52CEA050C304DA842B3
:1006E00002D100252EE050E02E4DA84201D1012577
:1006F00028E02D4DA84201D1022523E02B4DA84230
:1007000001D103251EE02A4DA84201D1042519E09C
:10071000284DA84201D1052514E0274DA84201D15A
:1007200006250FE0254DA84201D107250AE0244DFA
:10073000A84201D1082505E0224DA84201D1092592
:1007400000E00A25BD4045EA0C05C6F808542568B6
:100750004E689D43F60300D51D43256065684E68CD
:100760009D43B60300D51D436560DAF80050564638
:100770004F689D43FF0200D51D43356075684F6883
:100780009D43BF0200D51D437560521C102AFFF423
:1007900033AFBDE8F88F000080000058F4440258E1
:1007A000000002580004025800080258000C0258C9
:1007B000001002580014025800180258001C025879
:1007C00000200258002402580069084000D001208F
:1007D00070470AB1018370474183704701488068C0
:1007E0007047000014000024024881680278114418
:1007F0008160704714000024032010B500F058F801
:100800000F2000F007F808B1012010BD00F022F819
:10081000002010BD70B50D4D04464FF47A71287854
:10082000B1FBF0F00A490968B1FBF0F000F05AFCA6
:1008300048B9102C07D200222146501E00F018F8AB
:1008400000206C6070BD012070BD00001400002409
:10085000000000247047002809DB012100F01F027E
:1008600091404009800000F1E020C0F8001170477D
:100870000E4BF0B41B68C3F30223C3F10704042C2E
:1008800000D904241D1D072D01D2002300E0DB1E2A
:10089000012606FA04F56D1E0D409D409E40761E11
:1008A000164045EA0601F0BC00F014BE0CED00E075
:1008B000064A00F0070110684FF6FF03184040EAAF
:1008C0000120034908431060704700000CED00E070
:1008D0000000FA052DE9F047DFF8BC9104460E460A
:1008E000D9F8000000F00700B0420CD2D9F800108F
:1008F00021F007013143C9F80010D9F8000000F0D9
:100900000700B0427ED12078DFF89081800707D5BC
:10091000D8F80010E26821F00F011143C8F8001068
:100920002078C00762D0D8F80010A26821F4706166
:100930001143C8F8001059496068183902281CD0C2
:1009400003281DD0096801281DD04907002960DA55
:10095000524F083F396821F0070101433960FFF722
:100960003DFF0546606841F28831022813D0032814
:100970001ED001288A4627D034E009688903E5E7BC
:1009800009688901E2E7C905E0E7FFF727FF411B96
:10099000514501D923E08A463868C0F3C2000228D5
:1009A000F3D123E0FFF71AFF411B514501D916E0AF
:1009B0008A463868C0F3C2000328F3D116E0FFF777
:1009C0000DFF411B51450AD83868C0F3C200012809
:1009D000F5D10BE0FFF702FF411B514502D903207F
:1009E000BDE8F087386810F0380FF3D1D9F800105F
:1009F000484601F00701B1420DD9016821F0070115
:100A0000314300E005E00160006800F00700B042FB
:100A100001D00120E4E72078400707D5D8F800107E
:100A2000226921F070011143C8F8001020780107F5
:100A30001B4805D50168626921F07001114301600E
:100A40002178C90605D50168A26921F4E061114346
:100A500001602078800607D51149091D0868E26900
:100A600020F070001043086000F066F8D8F800101D
:100A70004FF4807292FAA2F201F47061B2FA82F23B
:100A8000D140084A515CC840074908600F20FFF771
:100A9000C1FE0020A4E700000020005218440258C4
:100AA0001C440258061600080000002410B5FFF789
:100AB00016FD08490968012292FAA2F201F00F011D
:100AC000B2FA82F2D140044A515CC840034908603E
:100AD00010BD000018440258061600080400002447
:100AE00010B5FFF7E3FF07490968102292FAA2F256
:100AF00001F07001B2FA82F2D140034A515CC84061
:100B000010BD00001C4402580616000810B5FFF77F
:100B1000CDFF074909684FF4807292FAA2F201F4FE
:100B2000E061B2FA82F2D140024A515CC84010BD85
:100B30001C440258061600083548F0B50068364DCA
:100B400010F03801334809D00411082904D0334E7D
:100B500010290BD018290BD02046F0BD2968890632
:100B6000FBD52968C1F3C101C840F0BD3046F0BDD6
:100B7000274918310A68096812F00302284BC1F3AB
:100B800005111B68274F03F001033F68DFED260ABC
:100B9000B7EE001AC7F3CC0717FB03F300EE103AC9
:100BA000224BB8EE400A06D0012A01D0022A2BD0EF
:100BB000B4FBF1F008E02A68920603D52A68C2F374
:100BC000C102D040B0FBF1F001EE900A1868B8EE17
:100BD000612AC0F3080001EE900A1868F8EE611A65
:100BE00040EE201A31EE810A22EE000AC0F34620C0
:100BF000401C00EE900AF8EE600A80EE201ABCEE6F
:100C0000C10A10EE100AF0BDB6FBF1F0DCE70000FF
:100C1000104402580090D0030044025840787D01EF
:100C20002C44025834440258000000393044025821
:100C30002DE9F05F04460078DFF8FC8341F2883943
:100C4000DFF8F8A3FE4DC0074ED0D8F8001040469C
:100C5000C1F3C20102291AD00068C0F3C200032800
:100C600005D1DAF8000000F0030002280FD0606818
:100C7000B0F5803F12D010B1B0F5A02F19D0286880
:100C800020F480302860286820F4802009E028685B
:100C9000800329D56068002874D025E0286840F4D6
:100CA00080302860606890B1FFF798FD06464F4697
:100CB00009E0286840F480202860EFE7FFF78EFD08
:100CC000801BB8427DD828688003F7D50CE0FFF779
:100CD00085FD06464F4604E0FFF780FD801BB842C5
:100CE000F0D828688003F7D42078D64F80075AD5EB
:100CF000D8F8001040464FF47C3B11F0380F13D069
:100D00000068C0F3C200032803D1DAF800008007AE
:100D10000AD0E068A8B3296821F0190101432960CD
:100D2000FFF75CFD06461DE02868400702D5E06835
:100D30000028B1D02868E16820F019000843286035
:100D4000FFF74CFD064604E0FFF748FD801B022834
:100D5000B8D828684007F7D507E0FFF73FFD801BAC
:100D60000228AFD828684007F7D538689BFAABF25D
:100D700020F47C312069B2FA82F29040014339605C
:100D800011E000E0AEE0286820F001002860FFF7E5
:100D900025FD064604E0FFF721FD801B022891D8BF
:100DA00028684007F7D42078C00655D5D8F8001039
:100DB00040464FF0F84BC1F3C201012917D000683B
:100DC00000E0EDE0C0F3C200032805D1DAF800002E
:100DD00000F0030001280AD0E069002828682CD020
:100DE00040F080002860FFF7F9FC064616E028680E
:100DF000C00502D5E069802874D138689BFAABF24F
:100E000020F0F841206AB2FA82F290400143396042
:100E100022E0FFF7E3FC801B022899D82868C00570
:100E2000F7D538689BFAABF2216AB2FA82F220F069
:100E3000F8409140084338600EE020F080002860C0
:100E4000FFF7CCFC064604E0FFF7C8FC801B022835
:100E500087D82868C005F7D42078000724D5774FB5
:100E600060694C37002838680FD040F001003860C6
:100E7000FFF7B4FC064604E0FFF7B0FC801B022835
:100E80008DD838688007F7D50EE020F00100386073
:100E9000FFF7A4FC064604E0FFF7A0FC801B022835
:100EA0007ED838688007F7D42078800623D5A069DB
:100EB000002828680FD040F480502860FFF78EFC8F
:100EC000064604E0FFF78AFC801B022868D82868E1
:100ED0008004F7D50FE020F480502860FFF77EFCF7
:100EE000064605E0D6E0FFF779FC801B022857D8BC
:100EF00028688004F7D42078400744D5524F3868DA
:100F000040F480703860FFF769FC064604E0FFF7A4
:100F100065FC801B642843D83868C005F7D5474F67
:100F2000A068483701280AD008B1052811D03868D0
:100F300020F001003860386820F0040002E03868D2
:100F400040F001003860A06888B1FFF747FC064612
:100F500009E0386840F004003860F0E7FFF73EFC35
:100F6000811B49451CD838688007F7D50BE0FFF78F
:100F700035FC064604E0FFF731FC811B49450FD8DC
:100F800038688007F7D4606AF0B3D8F80010C1F36E
:100F9000C20103297ED00228286820F0807000E07A
:100FA00079E0286003D0FFF719FC044687E0FFF7DB
:100FB00015FC064604E0FFF711FC801B02287BD8D5
:100FC00028688001F7D4DAF8001040F2F332914338
:100FD000E26A41EA0211A26A1143CAF8001094F8C9
:100FE00034004FF4FE02218E4002491EA0F500702D
:100FF00080B2C1F308010843218F491E02EA014172
:10100000084394F83C1000E05CE0491E120202EA3A
:10101000016108430949083108600B1D19684FF642
:10102000F872A06C914392FAA2F2B2FA82F2904066
:1010300001431960014809E010440258284402584D
:10104000004402580444025800480258001D016838
:10105000226C21F00C01114301600168626C21F0E7
:10106000020111430160016841F4803101600168AF
:1010700041F400310160016841F4802101600168A0
:1010800041F001010160286840F080702860FFF79E
:10109000A5FB01E018E00FE0044604E0FFF79EFB2B
:1010A000001B022808D828688001F7D50AE0FFF75E
:1010B00095FB001B022802D90320BDE8F09F286899
:1010C0008001F4D40020F8E70120F6E74FF0E0219A
:1010D0000428086903D020F004000861704740F03C
:1010E0000400FAE7401EB0F1807F10B501D3012063
:1010F00010BD4FF0E02460610F21601700F0EAF9A5
:101100000020A06107202061002010BD10B50068FC
:1011100086B01B49884230D11A48016841F001016C
:101120000160006800F00100059016481030016869
:1011300041F01001016000680121134C00F0100023
:1011400005904FF4007000900220CDE9010103905A
:101150000720694604902046FFF742FA4FF4806169
:10116000204600916946FFF73BFA2520FFF773FB05
:10117000032225201146FFF77BFB06B010BD0000BF
:1011800000100140E04402580000025830B50068E9
:10119000114988420CD1114A5088010408D41146E3
:1011A0004FF000034404097806D50A2901D0538082
:1011B00030BD40F400400DE00D2909D0084DC0F3CA
:1011C0000D04401C80B2C72829555080EFD830BD8F
:1011D00040F48040508030BD001001400C000024DD
:1011E0002400002454482DE9F041524C86B0016897
:1011F00041F002010160016841F0200101604E48A8
:101200000C38016841F480410160402000900220C8
:1012100001900320DFF82481002569460A270497FE
:10122000CDE902504046FFF7DBF904206946092664
:10123000049600904046FFF7D3F90496C020404E34
:10124000694600903046FFF7CBF94FF4407069468D
:10125000049700903046FFF7C3F9374864380168B7
:1012600041F480410160016821F48041016031480E
:10127000203881688906FCD43249016032494160D6
:10128000016841F00101016081688906FCD44FF4D6
:101290009C71416181688907FCD5C16841F00201F8
:1012A000C16081688906FCD44FF483714161816813
:1012B0008907FCD5C16841F00201C16081688906D7
:1012C000FCD422494161056181684907FCD5302180
:1012D0002170016841F00401016081688907FCD533
:1012E000C16841F00201C16081688906FCD481684F
:1012F0008906FCD4C561164941611648016821F48C
:1013000080310160134970310A6822F001020A60DD
:101310000A1D156082060F4B78331A601B1D0E4A9A
:101320001A6005220A60016841F48031016006B04C
:10133000BDE8F08120500052E044025800040258F9
:10134000001402581003000101041600C00300033A
:10135000EBEF180F24ED00E02D00030370B5294CCE
:101360009CB0256825F004052560264C00260C3429
:10137000256845F440452560256805F440451B95E2
:101380002568AD04FCD5012400940CAD039624041B
:10139000019402240994CDE90A410796082485E8BE
:1013A0000D00CDE910466846FFF742FC98B9FFF7FB
:1013B00019FF3F2013900320CDE9140640200101BE
:1013C000CDE91640CDE9180150201A90022113A84A
:1013D000FFF780FA10B101201CB070BD0A48016807
:1013E00041F0800101600848F430016841F00201D9
:1013F0000160006800F002001B90FFF7DDF800209C
:10140000EAE700000C480258004402581C480168F2
:1014100041F4700101601B49086840F00100086058
:10142000184A0020103210600A68174B1A400A60F0
:10143000144A18321060121D1060121D1060114AFB
:1014400028321060121D1060121D1060121D1060F5
:10145000121D1060121D1060121D1060121D106010
:101460000A6822F480220A6006496031086001207F
:101470000649C1F80801C006014980390860704773
:1014800088ED00E0004402587FEDF6EA008000514C
:1014900070B50D4D00240D48FFF726F802E0641CDE
:1014A000AC4204D80948FFF724F82028F7D10024DB
:1014B00002E0641CAC4206D8054901220348FFF74C
:1014C0001DF80028F5D170BDFFFF0100EC000024DD
:1014D0000C0000240907090E002804DB00F1E020BD
:1014E00080F80014704700F00F0000F1E02080F851
:1014F000141D70477047000010B504460420FFF724
:10150000E5FD0148046010BD0800002470B500240A
:1015100005464FF47A7603E0304600F005F8641C87
:10152000AC42F9D370BD000070B54FF0E02500214A
:101530006C69094AAB6912685043AA699A42FCD0A7
:1015400002D2A3EB020302E0A4EB020633441944E7
:1015500013468142F1D370BD080000240349CA69D3
:101560005206FCD5C2B20A85704700000010014047
:10157000FEF7DEFFFFF740F9042302220521A02039
:10158000FFF7ECFE4FF4C870FFF7B6FF4FF4E13001
:1015900000F018F8FEF7B7FFFEF7BAFF0648002282
:1015A0000221FFF716F94FF47A7404A0FEF7B5FF95
:1015B0002046FFF7ABFFF8E7000402584F4B0D0A37
:1015C000000000000B490A4A10B5C1E900200020C4
:1015D0008860C860086188610C2048610846FEF791
:1015E000A1FFBDE81040044901220248FEF786BF72
:1015F00000100140EC0000240C0000244FF040706B
:10160000E1EE100A7047000000000102030401022D
:10161000030406070809000038160008000000242B
:1016200024000000D40200085C16000824000024F6
:10163000AC0D0000F00200080090D0030090D00331
:101640000000000000000000000000000100000099
:0C1650001000000000000000010100007C
:0200000490006A
:100000000FB4044910B503AA029800F005F810BC1B
:100010005DF814FB10000024074B70B50D467B44BF
:1000200000F011F80446284600F020F810B14FF017
:10003000FF3070BD204670BD3B15007801694A1C39
:1000400002610878704700B58FB0CDE90131002119
:10005000059105497944CDE903101146684600F041
:1000600009F80FB000BD0000E5FFFFFF007B00F0C6
:10007000800070472DE9F04106460024D6E9017062
:10008000F5688046304603E04146B847641C304678
:10009000A8470028F8D12046BDE8F08140F2C95CAD
:1000A000C0F6000C604740F2E15CC0F6000C60470F
:1000B00040F6710CC0F6000C604740F6570CC0F6D5
:1000C000000C604741F20D5CC0F6000C604740F246
:1000D000C97CC0F6000C604740F2D37CC0F6000C2F
:1000E000604740F6393CC0F6000C604740F6AD2C46
:1000F000C0F6000C604741F20D1CC0F6000C6047D2
:1001000040F2E97CC0F6000C604740F2DD7CC0F6AE
:10011000000C604741F28D1CC0F6000C604740F2B5
:100120007B3CC0F6000C604740F6E12CC0F6000CAA
:10013000604740F60D3CC0F6000C6047FEE7704794
:100140000120FFF7ABBF4FF40050FFF7A7BF04201B
:10015000FFF7A4BF0820FFF7A1BF00002A4810B591
:1001600086B0016841F001010160016801F0010100
:100170000591016841F004010160016801F004018A
:100180000591016841F08001016000680124694621
:1001900000F0800005901D48CDE90040022002904B
:1001A0001B48FFF780FF600300901A486946CDE9BD
:1001B00001041948FFF777FF0C20009017486946A3
:1001C000FFF771FF002202210620FFF771FF0620D2
:1001D000FFF773FF012202210820FFF769FF0820C3
:1001E000FFF76BFF022209201146FFF761FF09208C
:1001F000FFF763FF032202212820FFF759FF282081
:10020000FFF75BFF06B010BDE0440258000011117B
:10021000000002580000211100080258001C02587A
:1002200010B528B190F83510022903D0802141651E
:10023000012010BD1D4A4FF4956301688C189C4243
:1002400007D8042280F83520086820F001000860F3
:1002500029E00C6824F00E040C6001680A440A6866
:1002600022F001020A60016E0A6822F480720A60BC
:1002700090F85C30012202FA03F10D4B1960D0E9CD
:1002800019134B60C16E31B10B6823F480730B609E
:10029000D0E91C134B60002180F8341080F8352021
:1002A000016D01B18847002010BD0000F0FFFDBFC7
:1002B0000454025870B504461420FFF703FF354E6E
:1002C000012C354D14D03548042C31D0082C46D0A3
:1002D0004FF400518C425CD13148FFF7F8FE002802
:1002E00057D1287880B30020287070B301221DE018
:1002F0002C480121FFF7EBFE01284AD1687840B174
:1003000000206870002807D04FF00000287034D11A
:1003100039E04FF00100F4E74FF00100F6E74FF04D
:1003200001013046FFF7D8FE2878DEE7022111E010
:100330000421FFF7CCFE00282BD1687830B10020D3
:10034000687028B1012204E021E01EE00120F7E7F7
:10035000002201213046BDE87040FFF7BDBE0821F4
:10036000FFF7B5FE002814D1687840B1002068700E
:10037000297831B10021297028B10122CFE701206D
:10038000F5E70121F7E70022C9E70022CEE70120C7
:10039000AAE770BD0004025820000024001C025887
:1003A000000802580000025810B5FFF79AFE0849ED
:1003B00009684FF4807292FAA2F201F47061B2FA05
:1003C00082F2D140034A515CC8400349086010BD25
:1003D00018440258061600080000002410B5FFF764
:1003E00085FE07490968102292FAA2F201F0700115
:1003F000B2FA82F2D140034A515CC84010BD0000FD
:100400002044025806160008364930B50A680968C3
:1004100012F00302344BC1F305311B68334C03F077
:1004200010032468DFED320AB7EE001AC4F3CC04DF
:1004300014FB03F300EE103A2E4BB8EE400A07D03F
:100440002D4C012A01D0022A4AD0B4FBF1F10BE075
:10045000244C283C22689506284A03D52468C4F316
:10046000C104E240B2FBF1F101EE901A1968B8EE56
:10047000612AC1F3080101EE901A1968F8EE611AB9
:1004800040EE201A31EE810A22EE000AC1F3462125
:10049000491C00EE901AF8EE600A80EE201AFCEE7D
:1004A000C10AC0ED000A1968C1F30641491C00EEFB
:1004B000901AF8EE600A80EE201AFCEEC10AC0ED38
:1004C000010A1968C1F30661491C00EE901AF8EEA2
:1004D000600A80EE201ABCEEC10A80ED020A30BD2F
:1004E000074ABFE7284402582C4402583C440258AB
:1004F000000000393844025800093D000090D00344
:1005000040787D01364930B50A68096812F0030267
:10051000344BC1F305511B68334C03F480732468DA
:10052000DFED320AB7EE001AC4F3CC0414FB03F378
:1005300000EE103A2E4BB8EE400A07D02D4C012A9F
:1005400001D0022A4AD0B4FBF1F10BE0244C283C44
:1005500022689506284A03D52468C4F3C104E24002
:10056000B2FBF1F101EE901A1968B8EE612AC1F3FD
:10057000080101EE901A1968F8EE611A40EE201A8F
:1005800031EE810A22EE000AC1F34621491C00EE39
:10059000901AF8EE600A80EE201AFCEEC10AC0ED57
:1005A000000A1968C1F30641491C00EE901AF8EEE2
:1005B000600A80EE201AFCEEC10AC0ED010A19683B
:1005C000C1F30661491C00EE901AF8EE600A80EE55
:1005D000201ABCEEC10A80ED020A30BD074ABFE70F
:1005E000284402582C440258444402580000003960
:1005F0004044025800093D000090D00340787D013E
:100600007047704790F8791090F87A000843704767
:1006100070B502680446D0691368916810F00F0F36
:1006200064D0594D03F490760D40354376D0C5071C
:1006300007D0DD0505D501251562E26F42F0010204
:10064000E267820708D5CA0706D0256802222A6217
:10065000E26F42F00402E267420708D5CA0706D0FB
:10066000256804222A62E26F42F00202E267020772
:100670000ED503F0200201F080552A4352EAC172E0
:1006800006D0256808222A62E26F42F00802E2677B
:10069000E26F002A3AD0800608D503F0200001F06E
:1006A0008051084302D0204600F0D1F9E06F0007E6
:1006B00003D42068806840062AD5204600F0B9F9A6
:1006C0002068816849061ED5816821F0400181605B
:1006D000606FC0B12D490165606FFFF7A1FD002873
:1006E00014D0606F016DBDE870400847850615D5D0
:1006F00003F0200501F0805635430FD02046BDE8B9
:10070000704000F0A4B92046FFF77BFF70BD05E004
:100710002046FFF776FF0020E067F7E7C6024FF0BC
:1007200020050CD54E020AD5E803106284F87950F2
:1007300084F87A502046BDE87040FFF761BF060696
:100740000AD503F0800601F400010E4304D02046D0
:10075000BDE8704000F00ABC41060BD5590609D52A
:100760001168204621F04001116084F8795000F0B2
:1007700097F8CBE70002C9D55800C7D5106820F01C
:1007800080401060C2E70000010000101F0A0090C6
:1007900010B5040003D094F8790010B107E00120EF
:1007A00010BD002084F878002046FFF7A4FC242028
:1007B00084F879002068016821F001010160204679
:1007C00000F080F90128EBD0606B10B1204600F0FA
:1007D00094F82068416821F4904141602068816864
:1007E00021F02A0181602068016841F00101016067
:1007F0002046BDE8104000F0E4B890F87A30202B95
:100800004CD1B9B1B2B190F87830012B46D0012368
:1008100080F878304166A0F86820A0F86A20FF22AE
:100820008168B1F5805F07D07F2351B1B1F1805F5E
:100830000CD010E001207047016921B940F2FF118E
:1008400007E0016909BBA0F86C2004E00169E1B18F
:100850003F21A0F86C100021C167222280F87A2085
:1008600080F8781001688A6842F001028A600168A5
:100870000A6892000CD50A6842F480720A60006827
:10088000816841F08051816006E0A0F86C30E2E7B9
:10089000086840F49070086000207047022070479C
:1008A0007047FEE7104810B586B0016841F00201BC
:1008B0000160006801210D4C00F00200059003204A
:1008C000CDE90001CDE9021069462046FFF7EBFBB8
:1008D000012220461146FFF7FFFB0122204602219C
:1008E000FFF7FAFB06B010BDE044025800040258BE
:1008F000704770477047FFF703BC90F83410C90782
:1009000006D001684A68836B22F400321A434A60B9
:1009100090F83410890706D501684A68C36B22F441
:1009200080321A434A6090F83410490706D50168AE
:100930004A68036C22F480221A434A6090F834100B
:10094000090706D501684A68436C22F400421A433D
:100950004A6090F83410C90606D501688A68836C2D
:1009600022F480521A438A6090F83410890606D522
:1009700001688A68C36C22F400521A438A6090F8B6
:100980003410490611D501684A68036D22F48012BB
:100990001A434A60016DB1F5801F06D101684A68AB
:1009A000436D22F4C0021A434A6090F834100906DD
:1009B00006D501684A68806D22F4002202434A602D
:1009C0007047F8B500250446C567FFF79EFB07464C
:1009D000206800686FF07E46000708D500223B467D
:1009E0004FF400112046009600F0FAFA60B9206832
:1009F000006840070AD500223B464FF4800120469C
:100A0000009600F0EDFA08B10320F8BD202084F82C
:100A1000790084F87A00002084F87850F8BD10B589
:100A2000806B0021A0F86A10A0F86210FFF7E9FDC2
:100A300010BD01680A6822F490720A6001688A6831
:100A400022F001028A60202180F87A10704710B5E8
:100A5000B0F86C2090F87A300168222B05D0088B12
:100A600040F008000883022010BD898C8368B3F52C
:100A7000805F01D103696BB11140426E531C436624
:100A80001170B0F86A10491E0904090CA0F86A1028
:100A900007D015E0436E11401980416E891C4166F4
:100AA000EFE701680A6822F490720A6001688A68B8
:100AB00022F001028A60202180F87A10FFF72AFBD9
:100AC000002010BD2DE9F04F044600688025FD4B45
:100AD0000021D4F810C087B0A6680F46D4F81C8057
:100AE00046EA0C06D4F814C0A26A4CEA080C46EA9E
:100AF0000C0632430668DFF8D0C306EA0C0616433C
:100B0000066020684268E66822F440523243426040
:100B10002268A0699A4201D0266A3043A66AB6F1DB
:100B2000005F04D1D4E90B6C46EA0C0630439668AA
:100B3000DFF898C306EA0C06064396602068C26A8E
:100B4000666A22F00F023243C262E14E2068E14A37
:100B5000B04210D1126802F03802182A74D005DCB5
:100B6000CAB3082A7AD0102A47D179E0202A7BD04C
:100B7000282A7CD17AE0D84EB04209D1126802F01E
:100B80000702062A73D2DFE802F053696B6D6F71BA
:100B9000D24EB04209D1126802F00702062A66D28C
:100BA000DFE802F0465C5E606264CD4EB04209D17F
:100BB000126802F00702062A59D2DFE802F0394F24
:100BC00051535557C74EB0420BD1126802F007027D
:100BD000062A4CD200E00EE0DFE802F02A40424450
:100BE0004648C14EB04209D1126802F03802182AB4
:100BF00038D0BBDCB4E74FF0010538E0BB4EB04263
:100C000009D1126802F00702062A30D2DFE802F0AA
:100C10001026282A2C2EB64EB0420BD1126802F0B4
:100C20000702062A23D2DFE802F003191B1D1F2149
:100C300000251CE098421AD1A64A121D126802F043
:100C40000702062A13D202E00CE007E00CE0DFE81E
:100C500002F0030507090B0D022508E0042506E054
:100C6000402504E0082502E0102500E02025DFF8FB
:100C700064B2A04E9842DFF880A2ABF1540B73D15E
:100C8000102D31D006DC022D09D0042D0AD0082DFC
:100C90002FD111E0202D29D0402D2AD107E0FFF7D8
:100CA0009DFB13E06846FFF7AFFB01980EE003A839
:100CB000FFF728FC049809E0DBF800105846890685
:100CC00010D50068C0F3C1012AFA01F0002811D044
:100CD0006168894601EB410181420AD8B0EB093FC6
:100CE00007D808E05046F3E78448F1E74FF40040A6
:100CF000EEE7012733E1102D4FF000084ED006DC5F
:100D0000022D0FD0042D15D0082D04D12DE0202D5B
:100D10004AD0402D13D00127794AA0F54071914265
:100D200070D9E6E7FFF75AFB626A0023414636F8BE
:100D300012200DE06846FFF767FB019803E003A867
:100D4000FFF7E0FB04980023616A36F8112019468A
:100D5000FFF7E5F962680902030241EA10615008F1
:100D6000181841EB080115E032E0DBF80010584696
:100D7000890609D500680023C0F3C1012AFA01F0F1
:100D8000616A36F8112015E0606A002336F81020F9
:100D900050460FE00023FFF7C2F9BDE7606A002369
:100DA00036F81020554805E0606A002336F8102018
:100DB0004FF400400021FFF7B2F90902020241EAB4
:100DC00010614FEA590010184A4641EB0801E1E76B
:100DD000E3694FF4004293424DD1082D23D005DC46
:100DE0008DB1012D12D0042D06D112E0102D35D079
:100DF000202D3AD0402D11D0012721F00F00C1F352
:100E0000420108435AE0FFF78FF916E0FFF791F926
:100E100013E06846FFF7F8FA01980EE003A8FFF721
:100E200071FB049809E0DBF800105846890608D5E4
:100E30000068C0F3C1012AFA01F0616A36F81110A6
:100E400010E0606A36F81010BAFBF1F041006068FB
:100E500001EB5001B1FBF0F081B2CEE7606A36F8E9
:100E600010102648B0FBF1F0F0E7606A36F8100089
:100E7000B2FBF0F0EAE7082D4AD00ADC0DB3012DF1
:100E800043D0042D7FF44DAF6846FFF7BDFA0198BB
:100E900009E0102D52D0202D55D0402DF2D103A8BD
:100EA000FFF730FB0498616A36F81110B0FBF1F1DE
:100EB000606801EB5001B1FBF0F080B22168C860BE
:100EC0004DE01FE0000C0058F369FFCFFFF4FF1165
:100ED00000100140544402580044004000480040C3
:100EE000004C0040005000400014014000780040D9
:100EF000007C0040441000900090D00300093D00A9
:100F0000FFFC0F00FFF710F9CDE7FFF712F9CAE772
:100F1000DBF80020594692060AD50968C1F3C102E0
:100F20002AFA02F1626A36F81220B1FBF2F20FE0FF
:100F3000616A36F81120BAFBF2F209E0616A36F80C
:100F400011200949F1E7616A36F81110B2FBF1F29C
:100F5000616802EB5102B2FBF1F189B2C16007B0E6
:100F60003846BDE8F08F000000093D0090F8791088
:100F7000212901D002207047B0F8621021B18168A8
:100F8000B1F5805F13D014E001680A68920004D5BF
:100F90008A6822F400028A6003E00A6822F0800274
:100FA0000A600068016841F0400101600CE00169DD
:100FB00061B1C16D4A1CC265026809781185B0F83B
:100FC0006210491EA0F8621000207047C16D0268CF
:100FD0000988C1F308011185C16D891CC165EEE75F
:100FE0002DE9F0411E46174688460446069D1CE042
:100FF000681C1AD025B1FFF788F8801BA84214D9C5
:101000002068016821F4D07101602068816821F0B6
:1010100001018160202084F8790084F87A000020A2
:1010200084F878000320BDE8F0812068C16938EABF
:10103000010004D00020B842DAD00020F3E70120FC
:10104000F9E7FEE7010002000400060008000A00BC
:0C1050000C001000200040008000000197
:040000050800029954
:00000001FF
